:020000040000FA
:1000000083018B018A018228F000030EF100830135
:10001000861B0F28663081000B110B102F2803144C
:100020000B190310A70DA60DA50DA40DA30DA20D70
:10003000C0302304FF3A031D3428F8302405F03A79
:10004000031D2E28271C2E2860142708AC00260824
:10005000AB002508AA002408A900A3010B10710E0B
:100060008300F00E700E0900A217220F2E28F03028
:100070002305E03A031D2E286014E0152708AC0084
:100080002608AB002508AA002408A9002308A80018
:100090002E2882070134023404340834103420340A
:1000A00040348034310880382B06F039031DAD2AE6
:1000B0002A083F393006031DAD2A2B080F3937189F
:1000C00010388207122A122A122A122A122A122AF7
:1000D000122A122A132A192A1F2A252A2B2A312AE0
:1000E000372A3D2A122A122A122A122A122A122AE0
:1000F000122A122A4C2A5C2A8C2A6A2A542A632A37
:10010000982A7B2A8501860107309F008316A0303C
:100110008600103085009F0100308C0088308100FF
:1001200083128C0131309000203084008001840AD9
:1001300050300406031D962888308B00AD011C2327
:10014000B71941230230D00060188F21E01BA4288A
:10015000D00B5F293608D0003718F028580859040A
:10016000031DBE28541CB828541053143208C00074
:10017000D41CBE28D410D3143208C1005A085B0422
:10018000031DCF28541DC828541153153308C2002D
:10019000D41DCF28D411D3153308C3001E295C0801
:1001A0005D04031DDF28541ED92854125316340849
:1001B000C400D41EDF28D412D3163408C5005E084C
:1001C0005F04031D1E29541FE928541353173508D3
:1001D000C600D41F1E29D413D3173508C7001E2903
:1001E000580859045A04031D0729541CFB285410AD
:1001F00053143208C000D41C0129D410D31433087E
:10020000C100541D0729541153153408C2005C085D
:100210005D045E04031D1E29541E12295412531638
:100220003208C400D41E1829D412D3163308C500CE
:10023000541F1E29541353173408C600580840068B
:10024000031926290130531CFF30D80759084106ED
:1002500003192E290130D31CFF30D9075A08420652
:10026000031936290130531DFF30DA075B084306B6
:1002700003193E290130D31DFF30DB075C0844061B
:10028000031946290130531EFF30DC075D0845067F
:1002900003194E290130D31EFF30DD075E084606E4
:1002A000031956290130531FFF30DE075F08470648
:1002B0000319A4280130D31FFF30DF07A428D2017F
:1002C0000F0C0E0CD5000310550C8F1880380F380A
:1002D000D500580703185214550859070318D214AB
:1002E00055085A070318521555085B070318D2150D
:1002F00055085C070318521655085D070318D216F7
:1003000055085E070318521755085F070318D217E0
:1003100052080F398500520E0F398600A42860104C
:100320008B13E019B729A90CAA0CAB0CAC0C031C5D
:10033000AD2AA90CAA0CAB0C0318AD2AA90CAA0C67
:100340000318AD2A2A082B062C06031DAD2A2A08FD
:100350000319A42AF039703A0319B02A2A08C039BF
:10036000803A031952282A0FAD2A8B170800E01192
:10037000A80CA90CAA0CAB0CAC0C031CAD2AA80C45
:10038000A90CAA0CAB0C0318AD2AA80CA90CAA0C3A
:100390000318AD2AA80CA90C0318AD2A29082A06AF
:1003A0002B062C06031DAD2A2908F039703A031DCF
:1003B000AD2AE01FF92A601FF72A60132B08FB0003
:1003C0002918092B2A087423E018092BA919EA29EE
:1003D000291D092B291DF829A91DF02A861A092B88
:1003E0006019FC2ABF230B23601360101C23092B08
:1003F000B923FB007B30840007302B0549202B1EDE
:10040000092AAB198004FF3AAB1D80052A08742322
:10041000E629000503190F2AAB19F42A092BAB1D95
:10042000F42A092B432AC101D310D410531C5414AD
:10043000432AC00153105410D31CD414432AC301BF
:10044000D311D411531D5415432AC2015311541111
:10045000D31DD415432AC501D312D412531E5416EA
:10046000432AC40153125412D31ED416432AC7017F
:10047000D313D413531F5417432AC60153135413D1
:10048000D31FD417432AE0138B17B71D0800530856
:100490005404FB003F30BF2BFF30C300DB00D315FB
:1004A000C20153115411132AFF30C700DF00D317C4
:1004B000C601531354132B2AC301DB01D311C2010C
:1004C00053115411192AC701DF01D313C601531365
:1004D0005413312AC301DB01D311C001531054104E
:1004E000D318531D742A432AC101C201D3105311DA
:1004F000D4145415432AC701DF01D313C401531286
:100500005412D31A531F852A432AC501C601D31298
:100510005313D4165417432AC301DB01D311C0016E
:10052000C1015310D3105410D410531D5415432A35
:10053000C701DF01D313C401C5015312D3125412F2
:10054000D412531F5417432A2B08031DAD2A6013DE
:10055000E017850186018B170800E0138B17080050
:10056000E01FF92A601FF72A60132B08FB002A08F6
:10057000F739753A0319D02A013A0319CE2A023AFB
:100580000319DE2A013A0319E22A2A0803392D0742
:100590007423E018092BAA1DF02AE62A1C30CB2A66
:1005A000AA1DD82AAB03AB0D2B0DFC39AD00092BCE
:1005B000AB03AB0D2B0DFC392D06F22A0630AA1D1C
:1005C000F02A092B0730AA1DF02AFF2A861A092BC8
:1005D0006019FC2ABF230B23601360101C23092B16
:1005E000B9232B06031D092B0B236013092B60175E
:1005F000092BE0136013092B073A031D092B213047
:100600002B06031D092B9A230B23601360101C2358
:10061000092B8B1708000F3085004F3086000630FD
:10062000C8000030132B142BFF3E031D142BC80BE6
:10063000122B8501860108000030B923B000083074
:10064000B923B100B10E31097039B1000230B923BC
:10065000F038B200B20E0330B923F038B300B30E55
:100660000430B923F038B400B40E0530B923F038A3
:10067000B500B50E2030B923B6002130B923B7003C
:1006800008003F30B923D3003208531C0301C000D7
:10069000320837183308D31C0301C1003308371858
:1006A0003408531D0301C200330837180F30D31D1F
:1006B0000301C300340837183208531E0301C40075
:1006C000340837183308D31E0301C500350837181E
:1006D0003408531F0301C600350837180F30D31FE5
:1006E0000301C700D4010800E0106011003A0319AB
:1006F0000034083A03190834143A03191C341E3A1A
:1007000003190234013A03190334073A0319043474
:10071000013A03190534253A03192034013A031923
:1007200021346015273A03190634013A03190734B6
:10073000E0147F340130FB000030BF230F30FB009A
:100740000230BF230330BF230430BF230530BF2353
:100750000030FB000830BF238030FB001C30BF237B
:100760002830FB002030BF230830FB002130BF239E
:10077000080083169B001C141A0883120800B92372
:100780007B06031908007B0883169A001C158B133F
:1007900055309D00AA309D009C148B171C119C188D
:0607A000CF2B83120800BC
:02400E00423F2F
:104200000100FF000F000F000F000F0014000D0051
:104210000000FF00FF00FF00FF00FF00FF00FF00A5
:104220003434733465346D34613466342D34503431
:1042300046343634323438348000FF00FF00FF004B
:04424000280008004A
:1042500046342E3443346134F1346134643461348F
:10426000323435342F34303433342F34303437341F
:02427E009900A5
:00000001FF
